:020000040000FA
:02000000402896
:1000800008308316810083128501831604308500B1
:100090008312860183160030860083128C018D0145
:1000A0008E018F010C0886000512000005160D0850
:1000B00086008510000085140E08860005100000DB
:1000C00005140F0886008511000085150C150C0815
:1000D0008600051200000516CA200C110C088600C7
:1000E000051200000516CA209520131E74289030B2
:1000F0001402031D86289520131E742814089200EC
:100100000310920D02308A00002A742880301402F5
:10011000031D74289520131E7428140892000310E0
:10012000920D03308A00002B74280519952807309A
:1001300097000000970B99280830950094010E3025
:1001400097000000970BA1280310940C0519941731
:10015000950B9F28131612309700970BAD28051D9D
:10016000131208000C0886000512000005167428FA
:100170000D08860085100000851474280E0886007E
:1001800005100000051474280F0886008511000072
:1001900085157428103098001030193010309A00EE
:0E01A0009A0BD028990BCE28980BCC2808007B
:100400001208820700000000742800007428000011
:10041000742800007428000074280000742800006C
:10042000742800007428000074280000742800005C
:10043000742800007428000074280000742800004C
:10044000742800007428000074280000742800003C
:10045000742800007428000074280000742800002C
:10046000742800007428000074280000742800001C
:10047000742800007428000074280000742800000C
:1004800074280000742800007428000074280000FC
:1004900074280000742800007428000074280000EC
:1004A00074280000742800007428000074280000DC
:1004B00074280000742800007428000074280000CC
:1004C00074280000742800007428000074280000BC
:1004D00074280000742800007428000074280000AC
:1004E0008C17B2280C17B2288C16B2280C16B2281A
:1004F0008C15B2280C15B2288C14B2280C14B22812
:100500008D17B8280D17B8288D16B8280D16B828DD
:100510008D15B8280D15B8288D14B8280D14B828D5
:100520008E17BE280E17BE288E16BE280E16BE28A1
:100530008E15BE280E15BE288E14BE280E14BE2899
:100540008F17C4280F17C4288F16C4280F16C42865
:100550008F15C4280F15C4288F14C4280F14C4285D
:10056000742800007428000074280000742800001B
:10057000742800007428000074280000742800000B
:1005800074280000742800007428000074280000FB
:0805900074280000742800002B
:10060000120882070000000074280000742800000F
:10061000742800007428000074280000742800006A
:10062000742800007428000074280000742800005A
:10063000742800007428000074280000742800004A
:10064000742800007428000074280000742800003A
:10065000742800007428000074280000742800002A
:10066000742800007428000074280000742800001A
:10067000742800007428000074280000742800000A
:1006800074280000742800007428000074280000FA
:1006900074280000742800007428000074280000EA
:1006A00074280000742800007428000074280000DA
:1006B00074280000742800007428000074280000CA
:1006C00074280000742800007428000074280000BA
:1006D00074280000742800007428000074280000AA
:1006E0008C13B2280C13B2288C12B2280C12B22828
:1006F0008C11B2280C11B2288C10B2280C10B22820
:100700008D13B8280D13B8288D12B8280D12B828EB
:100710008D11B8280D11B8288D10B8280D10B828E3
:100720008E13BE280E13BE288E12BE280E12BE28AF
:100730008E11BE280E11BE288E10BE280E10BE28A7
:100740008F13C4280F13C4288F12C4280F12C42873
:100750008F11C4280F11C4288F10C4280F10C4286B
:100760007428000074280000742800007428000019
:100770007428000074280000742800007428000009
:1007800074280000742800007428000074280000F9
:08079000742800007428000029
:02400E00F13F80
:00000001FF
